:020000020000FC
:1000000005C043C0189554C01895189505E007BB66
:1000100000E008BB01E003BF02E009BF03E005BF49
:1000200000E40BBF06B301FBEEF306B301FBEEF7F2
:1000300000E60ABF0DE001BD789403D014D0A89566
:10004000FCCF30FB7EF0042D083060F0073250F416
:10005000053110F4497F06C00B3110F0466002C034
:1000600042604B7F0895042F0670002319F400E0CE
:1000700008BB0AC041FB16F0C09801C0C09A42FB01
:1000800016F0C29801C0C29A08952FB640FB56F0F0
:10009000442450E052BF52E058BF316052E055BF97
:1000A000416004C03E7F53E055BF4E7F2FBE189580
:1000B0002FB630FB0EF4439431FB1EF4639409F425
:0600C00073942FBE189599
:00000001FF
